:020000040000FA
:06000000673002303A28CF
:08000800A000030EA100831209
:1000100005191028831601178312B23081002B288E
:1000200083160113831203140B190310A80DA90DD5
:10003000AA0DAB0DAC0DAC16FF302C02031D2B2806
:10004000FA302B02031D2B2831152A08AF0029088E
:10005000AE002808AD008B100B11210E8300A00EFE
:04006000200E090065
:0C007400203084008001840A80300402E7
:10008000031C3C281230B0006B2183160C30850510
:1000900087018312850187010730990000309A009B
:1000A000103083168E008312603083168F00831207
:1000B0000030831691009F008312C83083168100A0
:1000C000831231309000003083168C008312103080
:1000D0008B00831600309B001C141A088312BC008E
:1000E000851DDC21831610309B001C141A08831216
:1000F000BD008D2181018E018F010B118B100B1022
:100100008C018B179220311995204D21B30B90282B
:10011000031085190314B90DF03039020319F620C4
:100120000222822864003210080031110130B70029
:100130008B132030370783169B001C141A08831278
:10014000A4001030370783169B001C141A08831272
:10015000A300A6000230A6060030370783169B00D6
:100160001C141A088312A200A7000130A7068B17DF
:10017000321CC02822090339A200A309A409A50939
:1001800024082F02031DF02823082E02031DF02847
:1001900022082D02031DF02801303702031DD52847
:1001A0003D18D5283D143E14812102303702031D2D
:1001B000DE28BD18DE28BD143E148421033037022A
:1001C000031DE7283D19E7283D153E14872104301B
:1001D0003702031DF028BD19F028BD153E148A21F1
:1001E000B70A053037020318080098280130B60016
:1001F000B300B400B500B70085018701B1139220A8
:10020000B30B1C29031085190314B90DF030390202
:1002100003194329B41F8501B41F8701B40B1C299E
:100220003708B6080319B60003191A29FF308500EC
:100230008700B6039630B400311DFF283111321CFF
:1002400026292D090339AD00AE09AF092F1CFF285F
:100250008E018F010C1CFF280C102E1EFF288B1303
:1002600020303707BB002F08BA005621103037075F
:10027000BB002E08BA00562100303707BB002D08FE
:10028000BA0056218B1785018701B70AB6010530E0
:100290003702031CFF288D2108003E1C08003E1079
:1002A0001030BB003D08BA00562108008B133A08F5
:1002B00083161C159A0083123B0883169B00553049
:1002C0009D00AA309D009C1464009C1864291C1198
:1002D00083128B170800831620309B001C141A0809
:1002E0008312C10041080F39C200410E0F39C3000B
:1002F0000130C2080319C2000130C3080319C3004A
:1003000008000130BD0008000230BD0008000430C4
:10031000BD0008000830BD00080001303D0203198F
:10032000A02902303D020319AF2904303D02031910
:10033000BE2908303D020319CD290130BD003E140D
:100340005830D30005128512051485108714071143
:1003500007148712071687110A30D40008004230AC
:10036000D30005128512051085108710071107109C
:100370008712071287110130D40008000530D3001E
:1003800005128512051485148710071107108716AA
:10039000071687110A30D40008000F30D300051665
:1003A000851205108510871007150714871207128C
:1003B00087150A30D4000800B601B301B4013C1C13
:1003C000E429BC01BC14E629BC013C143C08B6007D
:1003D0006400EA29EB29EC29ED29EE293130B41B20
:1003E0008500B41F8501B30BE829B40BE82903107D
:1003F000B60CB608031DE8290030BB003C08BA0063
:10040000562108008F08031908008E018F01D008BB
:100410000319792AD00F0E2AF023792A501C42089A
:1004200050184308D107031C182AFF30D100F023CD
:1004300056180516D618851656190514D61985149A
:10044000561A8714D61A071557180714D71887167F
:1004500057190716D719871551080E020318482A8D
:1004600058180512D818851258190510D819851072
:10047000581A8710D81A071159180710D918871257
:1004800059190712D9198711FF30500203190800B2
:100490008F08031D0800922051080E02031C482AF1
:1004A00056180512D618851256190510D61985103A
:1004B000561A8710D61A071157180710D71887121F
:1004C00057190712D719871158180516D818851605
:1004D00058190514D8198514581A8714D81A0715ED
:1004E00059180714D918871659190716D9198715D5
:1004F0000800D50B08004630D500D40B08000130A9
:10050000D000D10001305302031D8D2AD615581694
:100510000F30D4000230D300080002305302031D14
:10052000982AD71459140A30D4000330D300080095
:1005300003305302031DA22AD6140530D400043020
:10054000D300080004305302031DBB2A561558146B
:10055000D81460308B1383169B001C141A08831266
:100560008B173D190130D400043084000530BC18CD
:100570004730D300080047305302031DC92A3D19F4
:10058000D0013D190800D9140130D4004830D300FF
:10059000080048305302031DD52AD7140130D40077
:1005A0000530840B4730D300080005305302031D8B
:1005B000F72A0130D400BC18EC2A3D19D0013D19AE
:1005C000D1013D1908005714D9140A30D40006305F
:1005D000BD184430D30008005714D9140A30D40091
:1005E0004930BD184430D30004308400080049303D
:1005F0005302031D012B58150130D4004A30D3009B
:1006000008004A305302031D0D2B56150130D4004B
:100610000630840B4930D300080006305302031D16
:10062000182BD61458150530D4000B30D300080011
:100630000B305302031D232B5614D8140A30D40058
:100640000C30D30008000C305302031D2E2BD7159D
:1006500059150A30D4000D30D30008000D30530274
:10066000031D382B56160530D4000E30D300080079
:100670000E305302031D512BD616D8155816703064
:100680008B1383169B001C141A0883128B17BD1939
:100690000130D400043084000F30BC184B30D3003C
:1006A00008004B305302031D5F2BBD19D001BD194B
:1006B0000800D9150130D4004C30D30008004C306C
:1006C0005302031D6B2BD7150130D4000F30840B60
:1006D0004B30D30008000F305302031D892B01302B
:1006E000D400BC18802BBD19D001BD19D101BD1992
:1006F00008005715D9150A30D4001030D30008006F
:100700005715D9150A30D4004D30D3000430840079
:1007100008004D305302031D932BD8160130D4002E
:100720004E30D30008004E305302031D9F2BD616C7
:100730000130D4001030840B4D30D300080010304D
:100740005302031DAA2B5616D8160530D4000130CB
:10075000D300080042305302031DB62BBC18D61438
:1007600056160130D4004330D30008004330530202
:10077000031DC42BBC18D81458160130D4004230C5
:10078000BD1C4530D300080044305302031DD12B5B
:100790005815D815591459150130D4004230D300DA
:1007A000080045305302031DDE2B5615561657140C
:1007B00057150A30D4005830D3000800583053027F
:1007C000031DED2BD61558161430D40004308400C8
:1007D0000630BC184930D30008000130D3000800AF
:1007E00056180516D618851656190514D6198514E7
:1007F000561A8714D61A071557180714D7188716CC
:1008000057190716D7198715D601D7015818051299
:10081000D818851258190510D8198510581A87103C
:10082000D81A071159180710D91887125919071221
:0A083000D9198711D801D901080079
:084000000600030004000700A4
:02400E00CC33B1
:10420000010078007A007C007E007B0079007F004E
:104210007D007A0078007E007C00FF00FF00FF0038
:104220000000F200F600FA00FE00F200F600FA00CC
:10423000FE00F200F600FA00FE00FF00FF00FF00A3
:10424000220005000500050005000900090009001D
:1042500009000D000D000D000D00FF00FF00FF0024
:10426000FF00FF00FF00FF00FF00FF00FF00FF0056
:10427000FF00FF00FF00FF00FF00FF00FF00FF0046
:10428000FF00FF00FF00FF00FF00FF00FF00FF0036
:10429000FF00FF00FF00FF00FF00FF00FF00FF0026
:1042A000FF00FF00FF00FF00FF00FF00FF00FF0016
:1042B000FF00FF00FF00FF00FF00FF00FF00FF0006
:1042C0003C00FF00FF00FF00FF00FF00FF00FF00B9
:1042D000FF00FF00FF00FF00FF00FF00FF00FF00E6
:1042E0001400FF00FF00FF00FF00FF00FF00FF00C1
:1042F000FF00FF00FF00FF00FF00FF00FF00DD00E8
:00000001FF
